:020000040800F2
:1000000000020020A50400081105000821050008D1
:10001000E9060008F90600080907000800000000CA
:100020000000000000000000000000004104000883
:100030001907000800000000250400080B02000852
:100040000B0200080B0200080B0200080B0200085C
:100050000B0200080B020008510F0008510F0008A6
:10006000510F0008510F0008510F00080B02000843
:100070000B0200080B0200086D0E00080B020008BE
:100080000B020008410E00080B0200080B020008DA
:100090000B0200080B0200080B020008510F0008B9
:1000A0000B0200080B0200080B0200080B020008FC
:1000B0000B0200080B0200080B0200080B020008EC
:1000C0000B0200080B0200080B0200080B020008DC
:1000D0000B0200080B020008350E0008610E000834
:1000E000510F00080B0200080B0200080B02000869
:1000F0000B0200080B0200080B0200080B020008AC
:100100000B0200080B0200080B0200080B0200089B
:100110000B0200080B0200080B0200080B0200088B
:100120000B0200080B0200080B0200080B0200087B
:100130000B0200080B0200080B0200080B0200086B
:100140000B0200080B0200080B0200080B0200085B
:100150000B0200080B0200080B0200080B0200084B
:100160000B0200080B0200080B0200080B0200083B
:100170000B0200080B0200080B0200080B0200082B
:100180000B0200080B02000800F0D6BA704700000E
:1001900070B50C46064600F073F9094B094A1D6814
:1001A0002C44944202D8084A944207D20C2333606C
:1001B0004FF0FF3500F06CF9284670BD1C60F9E780
:1001C0000002002000000220EC0C0020194610461E
:1001D00000F0BEBA1946104600F0C2BA13230360FD
:1001E0004FF0FF307047132303604FF0FF3070472C
:1001F000132303604FF0FF30704702294FF00003D4
:1002000003608CBF00200120704700F08DBA000011
:10021000114B70B500241C60104B114D18682E68EE
:1002200000F09CF80F4B53F820301B68A3F1080234
:1002300096420FD026B13179092904BF0A213171C4
:10024000092103F8041C33F9021C074B2A601980AA
:10025000012070BD204670BD2C0400202004002029
:10026000280400203404002024040020082930B58C
:1002700003791AD9082B14D842791A4B53F8225013
:1002800000F108047DB12D68856053F822502C6080
:1002900043F82240144A44790123A34014682343BD
:1002A0001360017130BD8460F2E7082BF9D94579FC
:1002B0000C4B53F825203AB11468A2420BBF002220
:1002C000246843F825201460427953F82230002B2B
:1002D000E7D1054C012303FA02F2236823EA020363
:1002E0002360DEE7340400202004002008B50A4B18
:1002F0001B681A79082A02D95B7983420AD900F06F
:10030000CAF818B1054B01221A6008BDBDE80840C3
:1003100000F080B808BD00BF280400202C04002095
:1003200008B500F0ADF8094B094A1B88094D1BB20E
:10033000002442F82340084A286813682146013BFC
:100340001360FFF793FF2C6000F060F82404002096
:100350007404002028040020300400200023C20779
:1003600001D51846704740080133F8E7134423F0DD
:10037000030310B54FF077321C1F43F8042C6207BB
:1003800042BF4FF0883243F8082CA3F108044FF025
:10039000807304E909000F4B44F80C3C002344F837
:1003A000103C032344F8143C2246022344F8183C32
:1003B000012344F81C3C42F8201D0B2342F8043D65
:1003C000013B032BFAD120466FF0020340F8443D75
:1003D00010BD00BF210300080548064A064B01680E
:1003E000914201D1984201D3181A70470430F6E7C0
:1003F00000000020FEE7FEE700020020EFF3088087
:1004000070470000004870470000002000F03CF8F2
:1004100001DFFEE7024A536843F0805353607047A0
:1004200000ED00E0EFF3098020E9F00F40F804ED63
:1004300002490968086000F003F800002804002061
:10044000FFF7E6FE04480068016801C9B1E8F00F53
:1004500081F309880047000028040020BFF34F8F74
:100460000549064BCA6802F4E0621343CB60BFF350
:100470004F8F00BFFDE700BF00ED00E00400FA056C
:10048000EFF3108072B6704762B6EFF310807047DA
:1004900080F310887047EFF30580C0B27047704753
:1004A0007047000008B5FFF7FAFF6A46114B124982
:1004B000934213D3114A124B12498B4211D3124B60
:1004C000124A0021934211D3FFF7EAFF00F052F9DC
:1004D00001F0B8FEBDE8084000F0A8B943F8041BDD
:1004E000E6E752F8040F43F8040BE6E743F8041B71
:1004F000E8E700BF00000020FEE7FEE7BC3B000885
:10050000000200202004002020040020EC0C002029
:1005100008B50249042000F04BF900BF4933000838
:100520000D490E4A0E4B6846904203D8984201D9B5
:10053000002102E009468D46012104207246024254
:1005400002D1EFF3088001E0EFF309802DE9F00F0D
:100550006B4600F007F800BF0002002000000220F8
:10056000600500202DE9F04F9A46494B8FB0934625
:100570009A6B03925A6B04929F6ADA6A05921A6B1D
:10058000DB6B0793434B06921A68434B9A4204462F
:10059000884602D0414801F0A1FFB8F1000F4ED0CB
:1005A0003F4801F09BFF00252E463E4801F096FF94
:1005B00039463D4801F01EFF05993C4801F01AFFFD
:1005C00006993B4801F016FF07993A4801F012FFDF
:1005D0003A0403D50399384801F00CFF3B0603D5D4
:1005E0000499364801F006FF354801F077FF594677
:1005F000344801F0FFFEB8F1000F1BD1324801F082
:100600006DFF3146314801F0F5FE6946304BC91A9D
:1006100003D549422F4801F0EDFE20468268C368A9
:1006200001698C4641698E46AD46514691E8F00F0E
:100630004168006801BE2849052000F0B9F894E837
:100640000E00E068D4F81C90089020690990606959
:100650000A9019F4007F2148A6690D930CBF04F19C
:10066000200504F124050C920B9101F037FF089B43
:1006700000930BA90EC91A4801F0BCFECDF80090FA
:1006800033460A9A0999174801F0B4FE8DE700BF76
:1006900000ED00E000000020FEE7FEE74231000828
:1006A000583100081D320008263200083632000892
:1006B00046320008563200086632000876320008DA
:1006C000863200088B3200089D320008CE320008C6
:1006D00058010020F6320008233300088731000853
:1006E000A2310008DF31000808B50249062000F0F9
:1006F0005FF800BF3633000808B50249072000F054
:1007000057F800BF1031000808B50249082000F072
:100710004FF800BF5533000808B50249092000F022
:1007200047F800BF2231000808B502490A2000F04E
:100730003FF800BF34310008034B044A4FF4E13165
:10074000002000F0B1BA00BF04020020750B0008C1
:100750000A460146014800F018BA00BF0402002012
:1007600010B50A460C460146002000F047FA204624
:1007700010BD000008B50121094800F087FB0121E8
:10078000084800F083FB0121074800F07FFB0121AE
:10079000064800F07BFBBDE8084000F035B900BF1B
:1007A0000D0C02400C0C02400E0C02400F0C0240DB
:1007B00008B50E4B1A680C469AB9012203281A6034
:1007C00003D171460A4801F015FE2146094801F09F
:1007D00011FE00F0E5FB084801F00CFE074801F0AF
:1007E00009FEFFF74DFE00F0FDF800BF38050020C0
:1007F0007B3300087F330008A73300089B330008D1
:1008000008B500F099FC034801F0F4FD00F088FC05
:10081000002008BDA933000808B5034C2368012057
:1008200000F072F9FAE700BF3C0600201FB5FFF7A1
:1008300027FE0E4B0E481B68029300240D4B0093BD
:100840000F220C234FF48071019400F055F80A4BED
:100850000A481B6802930A4B009307220C234FF4AB
:10086000C061019400F048F8FFF7D0FD18020020A5
:100870003C050020190800081C020020400600204A
:100880000108000808B5FFF7FBFD094B1B681A7942
:10089000082A07D95A79074B53F8221011B1096871
:1008A00043F82210FFF7F4FDBDE80840FFF7B2BDA2
:1008B000280400203404002038B50B79082B03D914
:1008C00008490320FFF774FF4C7901F1080203681F
:1008D00013B98B60026038BD13F8035CAC42F8D3E7
:1008E0001846F4E769330008031F53F8042F9A42AF
:1008F000FBD0181A704700000F2A2DE9F74F054664
:100900008B4691469A4633D810F003031BBFC3F1C0
:100910000403ED180B46CB1A303B23F003031AF007
:10092000080F05EB030419D02A46A24213D3019302
:10093000FFF7A6FD2949019B8046012251F822605C
:1009400017B2C6B10132212AF8D14046FFF7A0FD07
:100950006FF08A073DE012600432E6E72D60E6E7BB
:1009600001212046FFF782FC4046FFF791FD30E071
:100970006FF015072DE041F822400C98E7802A46D9
:100980000D99FFF7F3FC0E9B154AA3624FF0FF335E
:10099000E3611368206001331AF0010F6562C4F847
:1009A0002CB084F805902671A660E6602661666129
:1009B000A66126621360D3D10A212046FFF756FCB8
:1009C0001AF0040FD0D14046FFF762FD4846FFF70A
:1009D0008DFC384603B0BDE8F08F00BF74040020E2
:1009E0003004002008B5EFF30581C1F3080119B107
:1009F0001039044801F0FEFC00BE042000F084F829
:100A0000FBE700BFF633000810B53C4C00F0ECFBF0
:100A10000022A260236823F0867323F480332360CE
:100A2000E260236843F48033236023689803FCD595
:100A30004FF08051002000F027FB314A136843F447
:100A400000431360A36823F0F003A360A368A360CE
:100A5000A36823F46043A360A36843F40043A36046
:100A6000A36823F4E053A360A36843F4A053A360F6
:100A700000236360636843F480036360636843F04A
:100A800008036360636843F4A8436360636863605A
:100A9000636843F0E0636360236843F0807323601E
:100AA00002F5E43213689901FCD5164B0021196058
:100AB000196841F400711960196841F48061196086
:100AC000196821F00F011960196841F005011960DA
:100AD000936823F003039360936843F002039360E9
:100AE000064B19469A681207FCD51A6822F00102D3
:100AF0001A600B689B07FCD410BD00BF0038024091
:100B000000700040003C0240174B93F9001004288D
:100B100006D8DFE800F00307101C1C0000221A7042
:100B20000846704701221A70104A136923F0040323
:100B3000136130BFF4E702221A700D4A136823F0E4
:100B400003031360094A136943F00403F0E7032227
:100B50001A70074B1A6842F00E021A605A6842F483
:100B600080725A60EEE700BF2002002000ED00E036
:100B70000070004038B50446043000F0BEFA054667
:100B8000204600F00BFB284638BDF8B504460E465B
:100B90001746051D3A463146284600F099FA00B13D
:100BA000F8BD0121204600F0C9FAF3E7420901230C
:100BB00000F01F0003FA00F0014B43F822007047D9
:100BC00000E100E0024B1B680BB1FFF75BBE704712
:100BD0002C04002008B50B689B0608D5064B496815
:100BE00003EBC002C9B253F8303050689847BDE8F3
:100BF0000840FFF7E7BF00BF500C00202DE9F84385
:100C000006460C461546FFF746FCDFF8849078B19F
:100C100018235E43254459F80630AC4201D1BDE8A3
:100C2000F8831A681206FCD514F8012B5A60F4E711
:100C3000134F4FEA860847440121384600F07EFAF8
:100C4000182303FB06960F48F17C0F4A0729D8BFEB
:100C5000024601F00701102013FB0103D118ADB2C9
:100C6000CC604D60D158094841F00101D150404459
:100C7000012100F063FA3846BDE8F84300F08EBA6F
:100C8000480C00200060024000640240400C00203C
:100C900008340008034A182303FB00204168407C05
:100CA00000F0F2B90834000801282DE9F84F054694
:100CB0000C4600F2A78018214143544F07EB01086E
:100CC0007E58534941F8302001EBC0014FF0000934
:100CD0004B60504B43F820904F48012140F825903D
:100CE00000EB850000F02AFAD8F808B049465846CB
:100CF00000F0CCF8D8F80C900121484600F0C6F876
:100D000098F810A05846514600F0FAF85146484667
:100D100000F0F6F82846FFF7BDFF98F811302401DF
:100D2000002B4FD13D48B0FBF4F000F015FF80469A
:100D300001F0BAF884B2204600F012FF01464046A6
:100D400000F058FE4FF0834100F05EFF01F0ACF878
:100D5000240100F00F00A4B204438023B460736147
:100D60000023336142F20C03F360182303FB057385
:100D7000DC7C072C28DC4FF40011022000F084F901
:100D8000274A1820102104F0070310FB031300FB6F
:100D900005702449057D90F9120002EB030E41EA2B
:100DA0004561D150331DCEF808300023CEF8143001
:100DB000FFF7FCFE062C0EDC04F10B0040B2FFF73F
:100DC000F5FE0EE01848AEE74FF48001022000F077
:100DD0005BF9164AD5E7072C0AD1154B4FF40042B0
:100DE0005A60F36843F02003F3600020BDE8F88FF9
:100DF0000C2C02DC04F13000E0E70F2CF1DC04F1F4
:100E00003700DBE74FF0FF30BDE8F88F083400080B
:100E1000500C0020480C0020400C002080DE800296
:100E2000006002405004010000BD01050064024062
:100E300000E100E001490020FFF7CCBE0044004083
:100E400008B5054B05484FF40012DA6000F0A6F92A
:100E5000BDE80840FFF7B6BE00600240400C00202D
:100E600001490120FFF7B6BE0048004008B5054B18
:100E700005484FF000629A6000F090F9BDE8084024
:100E8000FFF7A0BE00600240440C0020F8B50D46FC
:100E90000126C0F3832120F00F0400F00F0706FAAB
:100EA00001F1022000F0F0F807FA06FE03232268A1
:100EB00003FA0EF3D84302402260226805F00301D2
:100EC00001FA0EF111432160E2681040E060E16830
:100ED000C5F3810202FA0EF20A43E2606268BE4084
:100EE00022EA060262606268C5F30015BD40154340
:100EF0006560A268B6B21343A36000206683F8BDA4
:100F000020F00F03F0B500F00F041D686700032602
:100F1000BE4025EA06051D601D680222072C02FA64
:100F200007F242EA050294BF002401241A6003EB91
:100F3000840300F007001A6A80000F24844022EA2C
:100F400004021A621A6A01FA00F010431862F0BD36
:100F50002DE9F0410F4D104F6E692A6800241640AC
:100F60004FF0010808FA04F31E4206D06B6107EB4C
:100F7000C40357F83420586890470134102CF1D13D
:100F8000064B1B681BB1BDE8F041FFF77BBCBDE819
:100F9000F08100BF003C0140600C00202C040020C8
:100FA0002DE9F04F2D4B2E4A1B882E492E48DFF895
:100FB000CC90DFF8CCA0DFF8CCB08BB00126ADF838
:100FC000243001F017FAFFF707FA0546FFF71AFA7F
:100FD0000446FFF713FA2A46009023464FF40071A7
:100FE000224801F007FA25EAE5754FF4007759F831
:100FF00026401CB394F80480E26A5AF82830606AEC
:10100000079317440692FFF76FFC069AB4F906108F
:10101000079B101A22680592626A04920390E26AA2
:1010200002926279019209AAB8F1080FC8BF013291
:1010300000920544A26A584601F0DCF90136212EDF
:10104000D5D10B4B02958DE888000A4A0A4819460B
:1010500001F0D0F90BB0BDE8F08F00BF38340008C4
:101060003A34000840340008453400088B34000846
:1010700011350008133500081735000874040020E6
:1010800024020020D5340008042808D8DFE800F046
:10109000030A0F1419000D4A136C19431164BFF3AE
:1010A0004F8F7047094B5A6C11435964F7E7074B50
:1010B0001A6B11431963F2E7044B5A6B11435963DE
:1010C000EDE7024B9A6B11439963E8E70038024061
:1010D00070B514461CB18568C3689D4201D1101BD0
:1010E00070BD86680568731C83604368013B3340AC
:1010F000013CEB5C01F8013BECE7C268436830B5AA
:101100008468121B9A4208D0C2680468013B1340ED
:10111000551CC560E154002030BD4FF0FF3030BD9C
:1011200000B50448A1B001F0D9F980226946002039
:1011300000F0AAF8883500087047000070B5044632
:101140000D46FFF79DF9236806463BB94FF0FF3384
:101150002360FFF79DF90125284670BDC5B10E4BF0
:101160001D6802212846FFF781F8236801330AD160
:1011700005F1080323600023AB603046FFF788F9D0
:10118000FFF748F9E7E729462046FFF795FBF4E724
:10119000FFF77EF9E0E700BF2804002070B50446A1
:1011A000FFF76EF9256806461DB9BDE87040FFF7E8
:1011B0006FB96B1C02D100232360F6E728460A2191
:1011C00050F808392360FFF751F8236813B94FF03E
:1011D000FF33236015F8034C3046FFF759F92046DA
:1011E000BDE87040FFF782B80F4BD3F8882042F477
:1011F000700210B5C3F888204FF000629A600B4C63
:10120000102283F822200021DA7760180131522958
:1012100080F80023F9D11A6942F010021A615A6964
:1012200042F400725A6110BD00ED00E000E100E000
:101230000C4B0146186882689368013B002B10B480
:10124000936005DA9469A34208DBCBB20A2B05D080
:101250001368581C1060197010BC704710BC01F066
:1012600055BA00BF5002002008B53E20FFF7E0FF4E
:101270002020FFF7DDFF034B1B689868BDE808409E
:1012800000F0E8BE500200202DE9804887B000AF92
:1012900081460E469346FFF7E7FFDFF858A2B046B7
:1012A0000BF1FF340025A8EB0603A3420BDA894BB0
:1012B000186841684B68013B002B4B6006DA01F06F
:1012C00015F9002806DAFFF7CFFFE8E70B685A1C8C
:1012D0000A6018780D2801D00A281BD100240D209F
:1012E00088F80040FFF7A4FF0A20FFF7A1FF46455A
:1012F000E9D033462246254620461978202930D9A0
:10130000222901D0272938D15C7804BB724801F02A
:10131000E5F8D8E7082801D07F2812D14645C2D089
:1013200008F1FF33082008F8015CFB60FFF780FF3D
:101330002020FFF77DFF0820FFF77AFFFB68984623
:10134000B1E708F10103FB6088F80000F4E75C2CCA
:101350000CD001331C788C42D6D159782029D5D8AD
:1013600001351978D1B103F8010BC6E79C1C9B78B5
:101370000132002BCAD02346ECE719785C290BD147
:10138000591C5B780132002BC0D04B1C49782229B4
:10139000BCD02029F1D8E3E71946F6E7002D92D01A
:1013A000AB000E3323F00703C7F80CD0ADEB030DF1
:1013B0006C464DF82510304690F800E003460130A9
:1013C000BEF1000FF8D0BEF1220F02D0BEF1270F00
:1013D00000D1013344F821301846013390F800E081
:1013E000BEF1000FF8D101318D42E5D1201F1AB1B5
:1013F00050F8043F002B3DD12268C7F81090C7F881
:1014000014A0002307F1100151F82380B8F1000F58
:101410003ED10133022BF5D12168304801F0D5F8D7
:101420000546002851D12E4A2E492F48DFF8B880B2
:1014300000F0E0FF2D4801F051F82C46C7F810905D
:10144000C7F814A007F1100353F8245025B10C3548
:101450000C3555F8181C91BB0134022CF2D12BE04D
:10146000BEF15C0F06D191F800E0BEF1000F08D18B
:10147000013AC1D0194613F801EBBEF1000FEFD1CC
:10148000B5E791F801E001F801EBECE708F10C0891
:10149000D8F800000028BCD011467B60BA6001F08B
:1014A00094F8BA687B680028F0D1D8F80830002B8F
:1014B000B2D0214628469847D7F80CD003E755F814
:1014C000142C404600F096FFC2E72168084800F05F
:1014D00091FFF1E75002002099350008B23500086D
:1014E000B7350008C3350008CB350008D5350008EE
:1014F000FD3500081C36000808B5FEF7AFFF0020D8
:1015000008BD08B5FFF74CFD002008BDF7B50C4637
:1015100005466946204600F0DDF9061E05DC294631
:101520000A4800F067FF03B0F0BDE368A768187AC7
:1015300000F04AF9294603463A46054800F05AFFAA
:10154000F1B2684600F0DCF8EDE700BF383800087B
:101550005F38000801282DE9F34105460C461EDCE2
:101560004A4B1C68BCB14A484A4F00F0B7FF0025FF
:10157000E368187A00F028F9A3680246294638463D
:1015800000F038FF24686E1C3546002CF0D1002096
:1015900002B0BDE8F081404800F0A0FFF7E73F4906
:1015A000606801F012F848BB022D05D194E80600EE
:1015B0003B4800F01FFFEAE73A49A06801F005F850
:1015C00070B9324B384D1C68002CE0D02146461CC7
:1015D000FFF79CFF284600F081FF24683046F3E7C0
:1015E000A06800F081FC044600F066F9014608B9E5
:1015F0002E48D1E72046FFF789FFC8E72C496068ED
:1016000000F0E3FF064600283CD1032D03DC94E8FC
:1016100006002848CDE7A06800F066FC074600F009
:101620004BF9804608B92448B6E708223146684697
:1016300000F02CFE062DD4BF033D0325083454F8DA
:10164000040F00F051FC2DF816000136AE42F6D121
:10165000D8F808201948394600F0CCFEF1B26846A7
:1016600000F04EF86946404600F03CF90028394643
:1016700006DC86300CBF1248124800F0BBFE86E73D
:101680001148FAE721681148F7E700BFE00C002095
:10169000C1360008E1360008D0360008EC360008F4
:1016A000F13600080F370008A83300081337000888
:1016B000343700083A3700087537000893370008B8
:1016C000AF370008D2370008F93700082238000881
:1016D0000238C0B211289ABF024B53F820000248CA
:1016E000704700BF7C380008A83300080F30C0B234
:1016F0001E289ABF014B185C00207047C4380008B0
:101700002DE9F74F0F46054608B1032905D92648AC
:1017100000F0E4FE03B0BDE8F08F2448DFF89C80C1
:10172000DFF89C90DFF89CA000F064FE2C460026B9
:10173000B742EFD095F90700FFF7D8FF314683464F
:10174000404600F057FEBBF1000F06D0B4F9001080
:1017500017485A4600F04EFE07E095F9072072B987
:10176000B4F90010134800F045FEA879FFF7B0FF68
:101770000146114800F03EFE01360234D8E7131D41
:10178000DBB2032B0CD8B4F900105242684600F0CB
:10179000D8F802AB1844694600F808BC5046E2E7A6
:1017A000B4F900104846D5E7E338000801390008CD
:1017B0000E39000819390008E83600080739000812
:1017C000163900081339000882283AD018D844285E
:1017D0002FD00CD8402828D003D8002841D0224848
:1017E0007047422823D04328F9D120487047462823
:1017F00023D020D3802822D08128F0D11C487047E4
:10180000872826D008D884281FD01CD385281ED02E
:101810008628E4D11748704789281ED01BD38A2810
:101820001DD0FF28DBD11448704714487047144876
:10183000704714487047144870471448704714485C
:10184000704714487047144870471448704714484C
:10185000704714487047144870471448704714483C
:1018600070471448704700BF113A000862390008F9
:1018700096390008CD390008073A00084E390008AB
:10188000563900086C39000876390008813900089B
:101890008C390008A0390008AB390008B5390008B8
:1018A000C1390008D7390008E2390008EE390008CC
:1018B000FA39000842390008054B1B6800228242B1
:1018C00000DA0BB9184670471B680132F7E700BF12
:1018D000E00C002018B1C36840681B6818476FF01F
:1018E0001200704718B1C36840685B6818476FF012
:1018F0001200704710B503460A4601200A24092A3F
:101900000DD85BB103440A24B1FBF4F204FB1211BD
:10191000303103F8011D1146002AF5D110BDB2FB8C
:10192000F4F20130EBE7002910B54FEAD17404DA84
:1019300010B12D23037001304942FFF7DBFF204433
:1019400010BD042A2DE9F74307460E4690464BD8B2
:1019500022B9FFF7E8FF03B0BDE8F08300291EDAE3
:10196000D8B12D2303700124764236B2002501231D
:101970000A216A1C904501FB03F312D196FBF3F197
:1019800009B211FB03F33819F61AFFF7CCFF36B290
:10199000204447B9AC1C2044DDE70446E4E70024BA
:1019A000E4E71546E5E7441C2E2304EB08050DF19A
:1019B00004083B5407EB000931464046FFF7B3FFEC
:1019C0004B462D1A3022AC4205D300223B198242ED
:1019D00005D1A018BFE7013403F8012FF3E718F889
:1019E000021099540132F2E70020B4E780F0004081
:1019F00002E000BF81F0004142001FBF5FEA4103E7
:101A000092EA030F7FEA226C7FEA236C6AD04FEAE6
:101A10001262D2EB1363C1BFD2184140484041402B
:101A2000B8BF5B42192B88BF704710F0004F40F4DD
:101A3000000020F07F4018BF404211F0004F41F4F9
:101A4000000121F07F4118BF494292EA030F3FD0C5
:101A5000A2F1010241FA03FC10EB0C00C3F12003D8
:101A600001FA03F100F0004302D5494260EB400067
:101A7000B0F5000F13D3B0F1807F06D340084FEAD2
:101A8000310102F10102FE2A51D2B1F1004F40EBC7
:101A9000C25008BF20F0010040EA0300704749002F
:101AA00040EB000010F4000FA2F10102EDD1B0FAFA
:101AB00080FCACF1080CB2EB0C0200FA0CF0AABFEF
:101AC00000EBC25052421843BCBFD040184370478D
:101AD00092F0000F81F4000106BF80F40000013293
:101AE000013BB5E74FEA41037FEA226C18BF7FEA6A
:101AF000236C21D092EA030F04D092F0000F08BFAC
:101B00000846704790EA010F1CBF0020704712F092
:101B10007F4F04D1400028BF40F00040704712F1D1
:101B200000723CBF00F50000704700F0004343F036
:101B3000FE4040F4000070477FEA226216BF08466C
:101B40007FEA23630146420206BF5FEA412390EA2F
:101B5000010F40F4800070474FF0000304E000BF25
:101B600010F0004348BF40425FEA000C08BF7047D6
:101B700043F0964301464FF000001CE050EA01029A
:101B800008BF70474FF000030AE000BF50EA0102AF
:101B900008BF704711F0004302D5404261EB41019C
:101BA0005FEA010C02BF84460146002043F0B643C1
:101BB00008BFA3F18053A3F50003BCFA8CF2083AE6
:101BC000A3EBC25310DB01FA02FC634400FA02FCEF
:101BD000C2F12002BCF1004F20FA02F243EB0200F6
:101BE00008BF20F00100704702F1200201FA02FC58
:101BF000C2F1200250EA4C0021FA02F243EB02004B
:101C000008BF20EADC7070474FF0FF0C1CEAD0528E
:101C10001EBF1CEAD15392EA0C0F93EA0C0F6FD04F
:101C20001A4480EA010C400218BF5FEA41211ED02D
:101C30004FF0006343EA501043EA5111A0FB013119
:101C40000CF00040B1F5000F3EBF490041EAD371EE
:101C50005B0040EA010062F17F02FD2A1DD8B3F16A
:101C6000004F40EBC25008BF20F00100704790F0D9
:101C7000000F0CF0004C08BF49024CEA502040EA2B
:101C800051207F3AC2BFD2F1FF0340EAC2507047F1
:101C900040F400004FF00003013A5DDC12F1190F2F
:101CA000DCBF00F000407047C2F10002410021FAA1
:101CB00002F1C2F1200200FA02FC5FEA310040F1B9
:101CC000000053EA4C0308BF20EADC70704792F032
:101CD000000F00F0004C02BF400010F4000F013A6A
:101CE000F9D040EA0C0093F0000F01F0004C02BF65
:101CF000490011F4000F013BF9D041EA0C018FE7D4
:101D00000CEAD15392EA0C0F18BF93EA0C0F0AD0D9
:101D100030F0004C18BF31F0004CD8D180EA0100FF
:101D200000F00040704790F0000F17BF90F0004F98
:101D3000084691F0000F91F0004F14D092EA0C0F7A
:101D400001D142020FD193EA0C0F03D14B0218BF0D
:101D5000084608D180EA010000F0004040F0FE4053
:101D600040F40000704740F0FE4040F440007047EF
:101D70004FF0FF0C1CEAD0521EBF1CEAD15392EA6E
:101D80000C0F93EA0C0F69D0A2EB030280EA010C5E
:101D900049024FEA402037D04FF0805343EA1111F7
:101DA00043EA10130CF000408B4238BF5B0042F155
:101DB0007D024FF4000C8B4224BF5B1A40EA0C00FA
:101DC000B3EB510F24BFA3EB510340EA5C00B3EB2C
:101DD000910F24BFA3EB910340EA9C00B3EBD10F1A
:101DE00024BFA3EBD10340EADC001B0118BF5FEA6C
:101DF0001C1CE0D1FD2A3FF650AF8B4240EBC25095
:101E000008BF20F0010070470CF0004C4CEA502055
:101E10007F32C2BFD2F1FF0340EAC250704740F4A4
:101E200000004FF00003013A37E792F0000F00F096
:101E3000004C02BF400010F4000F013AF9D040EA14
:101E40000C0093F0000F01F0004C02BF490011F4A8
:101E5000000F013BF9D041EA0C0195E70CEAD153A0
:101E600092EA0C0F08D142027FF47DAF93EA0C0F87
:101E70007FF470AF084676E793EA0C0F04D14B026B
:101E80003FF44CAF08466EE730F0004C18BF31F01D
:101E9000004CCAD130F000427FF45CAF31F0004317
:101EA0007FF43CAF5FE700BF42000ED2B2F1FE4FBD
:101EB0000BD34FF09E03B3EB126209D44FEA002319
:101EC00043F0004323FA02F070474FF000007047E0
:101ED00012F1610F01D1420202D14FF0FF30704781
:101EE0004FF00000704700BF0A22002100F0F8BB4D
:101EF0008A892DE9F041054610070C465AD44B68F3
:101F0000002B05DC0B6C002B02DC0020BDE8F0810F
:101F1000E66A002EF9D0002312F480522F682B605D
:101F200033D0606DA3895A0705D56368C01A636B07
:101F30000BB1236CC01A00230246E66A216A2846C8
:101F4000B047431CA38906D129681D294BD82B4AC9
:101F5000CA40D60747D500226260D90422692260B0
:101F600004D5421C01D12B6803B96065616B2F60F9
:101F70000029CAD004F14403994202D0284600F057
:101F80008DF900206063BDE8F081216A01232846B5
:101F9000B047411CC6D12B68002BC3D01D2B01D0EC
:101FA000162B01D12F60B0E7A38943F04003A38132
:101FB000BDE8F0810F69002FA7D093070E6808BF16
:101FC0004B690F6018BF0023A6EB07088B60B8F1C0
:101FD000000F9ADD43463A46216AA66A2846B04772
:101FE000002807DCA38943F04003A3814FF0FF30B2
:101FF000BDE8F0810744A8EB0008E8E701004020B5
:1020000038B50B6905460C46DBB118B183690BB9CD
:1020100000F072F80C4B9C4209D16C68B4F90C309A
:102020007BB121462846BDE83840FFF761BF074B2A
:102030009C4201D1AC68F1E7054B9C4208BFEC68BB
:10204000ECE7002038BD00BF403A0008603A0008C5
:10205000203A0008014620B9044B0549186800F0F1
:10206000D3B8044B1868FFF7CBBF00BF803A000815
:102070000120000850020020014900F0C5B800BF4F
:1020800001200008002310B504460360436083600C
:1020900081814366C28103614361836119460822DD
:1020A0005C3000F0F3F8054B6362054BA362054B0F
:1020B000E362054B2462236310BD00BF4525000881
:1020C000672500089F250008C325000870B54A1E33
:1020D000682555430E4605F1740100F02DF90446BC
:1020E00040B1002180E842000C30A06005F1680298
:1020F00000F0CCF8204670BD836910B5044633BBB0
:102100008364C3640365124B124A1B68826298425F
:1021100004BF0123836100F01FF86060204600F0D7
:102120001BF8A060204600F017F80022E0600421B0
:102130006068FFF7A7FF01220921A068FFF7A2FF4F
:1021400002221221E068FFF79DFF0123A36110BD69
:10215000803A000879200008F8B51C4B1E68B36966
:10216000074613B93046FFF7C7FF4836B4687368AF
:10217000013B03D5336833B13668F7E7B4F90C5047
:102180006DB16834F4E704213846FFF79FFF3060F3
:102190000028F1D10C233B6004462046F8BD4FF6E1
:1021A000FF73E3810123A38165662560A5606560F7
:1021B00025616561A5610822294604F15C0000F0F3
:1021C00065F86563A563A564E564E6E7803A000801
:1021D0002DE9F041884600F14804002614B9304644
:1021E000BDE8F081A5686768013F01D52468F5E77F
:1021F000AB89012B06D9B5F90E30013302D0284640
:10220000C04706436835EFE72DE9F8438046894625
:1022100000F14804002614B93046BDE8F883A568EB
:102220006768013F01D52468F5E7AB89012B07D921
:10223000B5F90E30013303D029464046C84706435E
:102240006835EEE770B50D4E0D4CA41BA4100025AB
:10225000A54209D10B4E0C4CFDF796FFA41BA41010
:102260000025A54205D170BD56F8253098470135A7
:10227000EEE756F8253098470135F2E7C03B0008F5
:10228000C03B0008C03B0008C03B000802440346B6
:10229000934200D1704703F8011BF9E738B50546B2
:1022A000002945D051F8043C0C1F002BB8BFE4189E
:1022B00000F062FB1F4A1368104633B96360146074
:1022C0002846BDE8384000F058BBA3420CD921682D
:1022D0006218934204BF1A685B68636004BF5218B7
:1022E00022600460ECE713465A680AB1A242FAD9A8
:1022F00019685818A0420BD120680144581882422E
:102300001960DDD1106852685A6001441960D7E73E
:1023100002D90C232B60D3E7206821188A4204BF1E
:1023200011685268626004BF091821605C60C7E7E9
:1023300038BD00BFE40C002070B5CD1C25F00305AE
:1023400008350C2D38BF0C25002D064601DBA942AF
:1023500003D90C233360002070BD00F00DFB234A2D
:102360001468214691B9224C23681BB93046FDF709
:102370000FFF206029463046FDF70AFF431C26D197
:102380000C233360304600F0F8FAE4E70B685B1B7F
:102390001AD40B2B0FD90B60CD50CC18304600F05F
:1023A000ECFA04F10B00231D20F00700C31A1BD028
:1023B0005A42E25070BD8C420DBF63684B68636047
:1023C000136018BF0C46E9E70C464968CAE7C41C0D
:1023D00024F00304A04205D0211A3046FDF7D8FEB0
:1023E0000130CDD02560D9E770BD00BFE40C0020DE
:1023F000E80C00200FB40A4B13B51C6824B1A36984
:1024000013B92046FFF778FE05AB049AA168019343
:10241000204600F0DBFA02B0BDE8104004B070477F
:102420005002002070B50E46054618B183690BB9FD
:10243000FFF762FEAB69AC6813B92846FFF75CFE94
:10244000234B9C4217D16C68A3891B071DD52369B8
:10245000DBB1013EA36816F8011F013BA360E9B997
:10246000002B2EDA22460A21284600F04FF90130CF
:1024700011D00A2070BD174B9C4201D1AC68E3E734
:10248000154B9C4208BFEC68DEE72146284600F069
:102490008FF90028DDD04FF0FF3070BD002B04DA3B
:1024A000A269934206DB0A2904D023685A1C2260E1
:1024B0001970CFE72246284600F028F90130C9D12B
:1024C000E9E723680A205A1C2260187070BD00BF1B
:1024D000403A0008603A0008203A0008024B0146E2
:1024E0001868FFF79FBF00BF5002002038B50C46A8
:1024F000054618B183690BB9FFF7FEFD0E4B9C42F0
:102500000DD16C682146284600F016FD88B9636835
:10251000013B636023685A1C2260187838BD074B62
:102520009C4201D1AC68EDE7054B9C4208BFEC68CA
:10253000E8E74FF0FF3038BD403A0008603A000845
:10254000203A000810B50C46B1F90E10FDF73EFE1A
:102550000028ABBF636DA3891B1823F48053ACBF65
:102560006365A38110BD2DE9F0411F468B89DB0512
:1025700005460C46164605D502230022B1F90E1079
:10258000FDF731FEA389B4F90E1023F48053A38123
:1025900032463B462846BDE8F041FDF71BBE10B56C
:1025A0000C46B1F90E10FDF71EFE431CA38915BFA2
:1025B000606523F4805343F48053A38118BFA38143
:1025C00010BDB1F90E10FDF709BE10F8012B11F87E
:1025D000013B012A28BF9A42F7D0D01A70472DE953
:1025E000F84F8046894692461F468B465D460A98BC
:1025F00015F8014B00F04AF92044467816F0080619
:102600000BD12D2C0BD12C7801260BF1020567B1D3
:10261000102F14D1302C0AD011E0AB46E6E72B2C5A
:1026200004BF2C780BF10205F1E7302C27D12B7871
:1026300003F0DF03582B4BD16C7810270235002EA6
:102640000CBF6FF000414FF000410022B1FBF7FEDC
:10265000104607FB1E1CA4F13003092B11D81C46A1
:10266000A7421DDD531C07D0864516D301D1A445D2
:1026700013DB00FB0740012215F8014BEBE70A27AB
:10268000DDE7A4F14103192B01D8373CE8E7A4F1B9
:102690006103192B04D8573CE2E74FF0FF32EBE718
:1026A000531C08D12223C8F800300846BAF1000FA5
:1026B00007D1BDE8F88F06B14042BAF1000F0CD047
:1026C00022B1013DCAF80050BDE8F88F4D46F9E748
:1026D0003024002FB3D10827B1E7BDE8F88F000000
:1026E000084B37B51C68084D236A002B08BF2B46E2
:1026F000009313460A4601462046FFF770FF03B0D9
:1027000030BD00BF50020020B4020020F8B50E46D4
:102710001446054618B183690BB9FFF7EDFC214B50
:102720009C422AD16C68A369A360A3891A072ED59D
:10273000236963B323692068C01A6369F6B29842BB
:10274000374604DB21462846FFF75AFC28BBA3681E
:10275000013BA36023685A1C22601E70636901302C
:10276000984204D0A389DB0719D50A2E17D1214638
:102770002846FFF745FC90B10FE00B4B9C4201D17E
:10278000AC68D0E7094B9C4208BFEC68CBE7214618
:10279000284600F00DF80028CCD04FF0FF3738461F
:1027A000F8BD00BF403A0008603A0008203A00082F
:1027B000324B70B51D6806460C4625B1AB6913B99E
:1027C0002846FFF799FC2E4B9C420FD16C68B4F958
:1027D0000C309AB215072CD4D00611D409223260DD
:1027E00043F04003A3814FF0FF3070BD254B9C4266
:1027F00001D1AC68EBE7244B9C4208BFEC68E6E7EC
:10280000510712D5616B41B104F14403994202D0E2
:102810003046FFF743FD00236363A38923F02403BD
:10282000A3810023636023692360A38943F0080325
:10283000A38123694BB9A38903F42073B3F5007F07
:1028400003D02146304600F049F8A28912F0010376
:102850000CD00023A36063695B42A361236953B971
:10286000B4F90C3013F08000BAD170BD920758BF94
:102870006369A360F2E70020F7E700BF5002002081
:10288000403A0008603A0008203A0008D0F8EC000E
:10289000704770B50E46B1F90E10002990B014467D
:1028A0001D4607DA00232B60B3891A0610D44FF4B3
:1028B00080630EE001AAFDF79BFC0028F2DB029A80
:1028C00002F47042A2F500535A425A412A60EEE7E0
:1028D00040230020236010B070BD00008B8973B5C9
:1028E0009D0706460C4607D504F147032360236184
:1028F0000123636102B070BD01AB6A46FFF7C9FFF7
:10290000009905463046FFF717FD38B9B4F90C3089
:102910009A05EFD443F00203A381E5E70C4BB362C1
:10292000A389206043F08003A381009B6361019B26
:1029300020614BB1B4F90E103046FDF75EFC18B1C2
:10294000A38943F00103A381A3891D43A581D1E796
:102950007920000882B001B901A942B14BB11378C6
:102960000B601278101C18BF012002B0704710468F
:10297000FBE76FF00100F8E7704770479368013B91
:10298000002B10B4936008DA9469A34202DBCBB247
:102990000A2B02D110BCFFF7B9BE1368581C106097
:1029A0001970C8B210BC7047F8B506460F461446F9
:1029B000D518AC4201D1002007E03A4614F8011BBB
:1029C0003046FFF7DBFF431CF3D1F8BD2DE9F04F94
:1029D0009DB00C4617460393064618B183690BB9A0
:1029E000FFF78AFB7C4B9C4257D17468A389180778
:1029F0005DD52369002B5AD00023099320238DF83D
:102A0000293030238DF82A304FF0010BB846454667
:102A100015F8013B002B55D1B8EB070A0BD05346F4
:102A20003A4621463046FFF7BFFF013000F0C48030
:102A3000099B5344099398F80030002B00F0BC80A8
:102A400000234FF0FF3204930793059206938DF80D
:102A500053301A9305222978604800F009FB05F1EC
:102A60000108049B002831D1D90644BF20228DF8EB
:102A700053201A0744BF2B228DF853202A782A2A84
:102A80002CD0079A00210A20A846013598F800307A
:102A9000303B092B6DD971B326E0514B9C4201D1DB
:102AA000B468A3E74F4B9C4208BFF4689EE72146F9
:102AB0003046FFF77DFE00289ED04FF0FF301DB05E
:102AC000BDE8F08F252BA7D0A846A0E7434A801A7F
:102AD0000BFA00F0184304904546BBE7039A111D1A
:102AE00012680391002A01DB079204E0524243F08E
:102AF00002030792049398F800302E2B10D198F817
:102B000001302A2B08F1010137D1039B1A1D1B68E4
:102B10000392002BB8BF4FF0FF3308F10208059372
:102B2000314D98F800100322284600F0A1FA40B178
:102B30004023401B03FA00F0049B0343049308F175
:102B4000010898F8001029488DF82810062208F18D
:102B5000010700F08DFA002834D0254B03BB039BFE
:102B6000073323F0070308330393099B4B4409936E
:102B70004CE700FB0232012186E70023059318464B
:102B80000A258846013198F80020303A092A03D9ED
:102B9000002BC5D00590C3E705FB00200123F0E71B
:102BA00003AB00932246134B04A93046AFF30080D9
:102BB000B0F1FF3F8146D8D1A3895B063FF57DAFD9
:102BC00009987CE703AB009322460A4B04A93046E0
:102BD00000F088F8ECE700BF403A00088A3A0008A5
:102BE000603A0008203A0008903A0008943A000839
:102BF00000000000A92900082DE9F04791461F4672
:102C00008A680B69DDF820809342B8BF1346C9F883
:102C1000003091F8432006460C4612B10133C9F842
:102C200000302368990642BFD9F800300233C9F852
:102C30000030256815F0060507D104F1190AE3688C
:102C4000D9F800209B1A9D4229DB94F84330226872
:102C5000003318BF012392062ED404F143023946F3
:102C60003046C047013021D02368E568D9F80020FC
:102C700003F00603042B08BFAD1AA36822690CBF3A
:102C800025EAE57500259342C4BF9B1AED184FF065
:102C900000091A344D451BD10020BDE8F0870123FF
:102CA000524639463046C047013003D14FF0FF301D
:102CB000BDE8F0870135C2E7E1185A1C302081F8E1
:102CC0004300224494F8451082F843100233C4E7CD
:102CD0000123224639463046C0470130E6D009F18B
:102CE0000109D7E72DE9F04317460A7E85B06E2A21
:102CF000984606460C460C9B01F1430E00F0BC8042
:102D00001AD8632A2ED00AD8002A00F0C880582A80
:102D100000F08A8004F1420584F842202AE0642A07
:102D200001D0692AF6D121681A6811F0800F23D0EA
:102D3000111D1960136827E0732A00F0B48008D8C9
:102D40006F2A2AD0702AE5D10A6842F020020A6070
:102D500003E0752A21D0782ADCD1782284F8452036
:102D60006E4964E01A6801F14205111D196013688B
:102D700084F842300123A3E011F0400F02F1040176
:102D80001960D7D0B2F90030002B03DA2D225B4254
:102D900084F8432062490A2217E02068196810F07D
:102DA000800F03D0081D18600B6806E010F0400F7C
:102DB00001F104001860F7D00B8859496F2A14BF3D
:102DC0000A220822002084F843006568A560002DCF
:102DD000C0F29C80206820F004002060002B3FD1CE
:102DE000002D40F095807546082A0BD12368DA073C
:102DF00008D5236962689A42DEBF302305F8013C9A
:102E000005F1FF35AEEB05032361CDF800803B46AD
:102E100003AA21463046FFF7EFFE013055D14FF0AF
:102E2000FF3005B0BDE8F08381F845203C492268B9
:102E3000186812F0800F00F104051D6001D00368CE
:102E400002E05506FBD50388D00744BF42F02002BC
:102E500022601BB9226822F0200222601022B1E712
:102E60007546B3FBF2F002FB1033CB5C05F8013D75
:102E700003460028F5D1B7E708681A68496910F0D9
:102E8000800F04D0101D18601368196007E010F05F
:102E9000400F02F1040018601368F6D01980002377
:102EA00023617546B1E71A68111D196015686268DB
:102EB0000021284600F0DCF808B1401B6060636820
:102EC0002361002384F843309FE723692A4639466B
:102ED0003046C0470130A2D023689B0707D50025A4
:102EE00004F11909E368039A9B1A9D4205DBE06827
:102EF000039B9842B8BF184693E701234A463946D8
:102F00003046C04701308AD00135EBE7002BA7D10E
:102F10000B7884F8423004F1420565E7AC3A0008CA
:102F20009B3A0008838903F00903092B01D1FFF7BD
:102F300091B8002070470000F8B50C46054618B15E
:102F400083690BB9FFF7D8F83B4B9C420AD16C68F8
:102F5000B4F90C200023636093B29E060CD54FF0A9
:102F6000FF30F8BD354B9C4201D1AC68F0E7344BE3
:102F70009C4208BFEC68EBE7580748D4D90605D453
:102F8000092342F040022B60A281E8E71A070BD523
:102F900021462846FFF734F80028E0D1A389A06035
:102FA00023F00803A381A061A38943F00403A38154
:102FB00023691BB921462846FFF790FCB4F90C7031
:102FC000BEB2B3070FD00123A3811E4B1E49186860
:102FD00006F00906FFF7FCF8092EA78103D1214668
:102FE0002846FEF785FF22692260666A6369216AC6
:102FF0002846B047002860601CDCA38917BF002268
:1030000043F0200343F040036260A381A7E7616BB4
:103010000029CDD004F14403994202D02846FFF79D
:103020003DF9236C636000206063002BC0D0E36B2C
:103030002360F8BD0020F8BD403A0008603A00085F
:10304000203A0008803A0008252F000849B1FF2ADD
:1030500085BF8A2303600A704FF0FF3098BF0120BC
:1030600070470846704700000000000000000000A4
:1030700001F0FF01102A2BDB10F0070F08D010F829
:10308000013B013A8B422DD010F0070F42B3F6D12D
:10309000F0B441EA012141EA014122F007047FF046
:1030A00000070023F0E80256083C85EA010586EA9D
:1030B000010685FA47F5A3FA87F586FA47F6A5FAD9
:1030C00087F68EB9EED1F0BC01F0FF0102F00702E5
:1030D00032B110F8013B013A83EA010313B1F8D190
:1030E0000020704701387047002D06BF3546033871
:1030F000073815F0010F07D1013015F4807F02BFAA
:10310000013015F4C03F0130F0BC0138704700BFFA
:10311000425553204641554C542048414E444C455D
:1031200052004445425547204D4F4E2048414E44A1
:103130004C45520044554D4D592048414E444C4554
:1031400052000A49535220737461636B206F766595
:1031500072666C6F77656400537461636B20706F87
:10316000696E74657220636F727275707465642C19
:1031700020726573657420746F20746F70206F66A1
:1031800020737461636B000A436F6E7465787420FA
:103190006265666F726520686172646661756C74E1
:1031A0003A0020202072303A2030782530386C7870
:1031B0000A20202072313A2030782530386C780A85
:1031C00020202072323A2030782530386C780A205E
:1031D000202072333A2030782530386C780A00206D
:1031E000207231323A2030782530386C780A20202D
:1031F000206C723A2030782530386C780A202020F4
:1032000070633A2030782530386C780A202070734B
:10321000723A2030782530386C780A0A00465352CA
:103220002F4641523A0020434653523A20307825E7
:1032300030386C780A0020484653523A20307825BE
:1032400030386C780A0020444653523A20307825B2
:1032500030386C780A0020414653523A20307825A5
:1032600030386C780A0020424641523A20307825A6
:1032700030386C780A004D4D4641523A203078255E
:1032800030386C780A004D697363004558435F52CB
:1032900045543A2030782530386C780A00417474EF
:1032A000656D7074696E6720746F207265636F6EF0
:1032B00073747275637420737461746520666F72C1
:1032C00020646562756767696E672E2E2E00496EF1
:1032D000204744423A0A2020736574202470633DDD
:1032E0003078256C780A20206672616D6520300A7E
:1032F000202062740A000A49535220737461636B80
:10330000206F766572666C6F7765642062792061E4
:1033100074206C6561737420256420627974657310
:103320002E0A0048415244204641554C5420484101
:103330004E444C4552004D454D204D414E41474570
:103340002048414E444C4552004E4D492048414E84
:10335000444C4552005553414745204641554C5435
:103360002048414E444C4552004641494C4544207A
:10337000415353455254494F4E2E0025700A002A9E
:103380002A2A2052494F54206B65726E656C20705A
:10339000616E69633A0A25730A0A002A2A2A20689C
:1033A000616C7465642E0A0A006D61696E28293AA1
:1033B00020546869732069732052494F5421202892
:1033C00056657273696F6E3A20323031372E303164
:1033D0002D646576656C2D3235352D673166623228
:1033E000312D56616E64726973290A0069646C65D7
:1033F000006D61696E00496E73696465206973725E
:103400002025640A00000000004400400000020083
:1034100003000240020002400700260604000000EC
:103420000048004000000400090C0240080C024063
:1034300007002703040000005F5173746174650086
:103440006E616D650009706964207C20252D323124
:10345000737C20252D397351207C20707269207C6B
:1034600020737461636B2028207573656429207C48
:103470002062617365202020202020207C2063753D
:103480007272656E74202020200A000920202D20F1
:103490007C206973725F737461636B20202020202D
:1034A000202020202020207C202D202020202020B3
:1034B00020202D207C2020202D207C2025356920D7
:1034C0002825356929207C2025313070207C202555
:1034D0003130700A000925336869207C20252D329F
:1034E0003073207C20252D387320252E3173207CCD
:1034F00020253369207C2025356920282535692938
:10350000207C2025313070207C2025313070200A2D
:10351000007C0053554D000925357320252D32318F
:10352000737C253133732536732025356920282592
:103530003569290A0073746F7070656400736C6577
:103540006570696E6700626C206D757465780062E5
:103550006C20727800626C2073656E6400626C206F
:103560007265706C7900626C20616E79666C0062C5
:103570006C20616C6C666C0072756E6E696E6700B3
:1035800070656E64696E670057656C636F6D65206A
:10359000746F2052494F5421007368656C6C3A2057
:1035A000696E636F72726563742071756F74696E92
:1035B000670068656C700044657363726970746954
:1035C0006F6E00436F6D6D616E6400252D32307338
:1035D0002025730A002D2D2D2D2D2D2D2D2D2D2D3A
:1035E0002D2D2D2D2D2D2D2D2D2D2D2D2D2D2D2D0B
:1035F0002D2D2D2D2D2D2D2D2D2D2D2D007368656F
:103600006C6C3A20636F6D6D616E64206E6F742018
:10361000666F756E643A2025730A00004C36000808
:1036200053360008F91400082C39000863360008E6
:10363000031500088D36000892360008551500085D
:103640000000000000000000000000007265626FD2
:103650006F74005265626F6F7420746865206E6FBE
:103660006465005072696E747320696E666F726D66
:103670006174696F6E2061626F75742072756E6E11
:10368000696E6720746872656164732E007361757A
:103690006C00696E74657261637420776974682068
:1036A00073656E736F727320616E642061637475ED
:1036B00061746F7273207573696E67205341554C46
:1036C00000494409436C61737309094E616D6500DB
:1036D0004E6F206465766963657320666F756E64EE
:1036E000002325690925730925730A007265616441
:1036F0000075736167653A202573202573203C644B
:1037000065766963652069643E7C616C6C0A006162
:103710006C6C006572726F723A20756E64656669D2
:103720006E656420646576696365206964206769F5
:1037300076656E0077726974650075736167653AC6
:10374000202573202573203C6465766963652069B4
:10375000643E203C76616C756520303E205B3C7693
:10376000616C756520313E205B3C76616C7565202F
:10377000325D5D0A006572726F723A20756E646523
:1037800066696E656420646576696365206769763D
:10379000656E0057726974696E6720746F20646586
:1037A0007669636520232569202D2025730A00652D
:1037B00072726F723A2064657669636520232569A9
:1037C000206973206E6F74207772697461626C6512
:1037D0000A006572726F723A206661696C75726573
:1037E00020746F20777269746520746F2064657629
:1037F000696365202325690A00646174612073751B
:10380000636365737366756C6C7920777269747421
:10381000656E20746F206465766963652023256971
:103820000A0075736167653A2025732072656164CB
:103830007C77726974650A006572726F723A2066ED
:1038400061696C656420746F2072656164206672C2
:103850006F6D20646576696365202325690A0052CF
:10386000656164696E672066726F6D20232569202B
:103870002825737C2573290A000000001C390008E4
:1038800020390008243900082639000829390008A1
:10389000A8330008A8330008863500082B39000833
:1038A000D53900082F3900083139000833390008AC
:1038B000363900083A3900083D390008A8330008B5
:1038C000403900086600007000006E0000750000BE
:1038D0006D00000000006B00004D00004700005428
:1038E000000050556E61626C6520746F20646973CE
:1038F000706C61792064617461206F626A656374C1
:1039000000446174613A00095B25695D2000256906
:10391000256300257300256945256900C2B0430071
:10392000C2B046004B006C78006D006470730041BB
:1039300000560047730042617200506100636400EA
:103940002500434C4153535F554E44454600414387
:10395000545F414E59004143545F4C45445F5247C8
:1039600042004143545F534552564F004143545F18
:103970004D4F544F52004143545F535749544348AD
:10398000004143545F44494D4D45520053454E5309
:10399000455F414E590053454E53455F42544E00DA
:1039A00053454E53455F54454D500053454E534586
:1039B0005F48554D0053454E53455F4C4947485469
:1039C0000053454E53455F414343454C0053454EDC
:1039D00053455F4D41470053454E53455F4759524C
:1039E0004F0053454E53455F434F4C4F5200534594
:1039F0004E53455F50524553530053454E53455F18
:103A0000414E414C4F4700434C4153535F414E5947
:103A100000434C4153535F554E4B4E4F574E0000A1
:103A20000000000000000000000000000000000096
:103A30000000000000000000000000000000000086
:103A40000000000000000000000000000000000076
:103A50000000000000000000000000000000000066
:103A60000000000000000000000000000000000056
:103A70000000000000000000000000000000000046
:103A800054020020504F53495800232D302B200062
:103A9000686C4C0065666745464700303132333408
:103AA00035363738394142434445460030313233A8
:103AB000343536373839616263646566000020202A
:103AC00020202020202020282828282820202020CE
:103AD000202020202020202020202020202088108E
:103AE00010101010101010101010101010100404EE
:103AF00004040404040404041010101010101041F5
:103B00004141414141010101010101010101010165
:103B100001010101010101010110101010101042FA
:103B20004242424242020202020202020202020235
:103B30000202020202020202021010101020000013
:103B40000000000000000000000000000000000075
:103B50000000000000000000000000000000000065
:103B60000000000000000000000000000000000055
:103B70000000000000000000000000000000000045
:103B80000000000000000000000000000000000035
:103B90000000000000000000000000000000000025
:103BA0000000000000000000000000000000000015
:103BB0000000000000000000000000000000000005
:103BC000F00C002000000000F8040020400000007D
:103BD0000000000000000000EC330008F133000892
:103BE000FF000000353500083D3500084635000867
:103BF0004F350008553500085D350008663500086A
:103C00006F35000800000000783500088035000896
:103C10005402002000000000403A0008603A00080A
:103C2000203A000800000000000000000000000032
:103C30000000000000000000000000000000000084
:103C40000000000000000000000000000000000074
:103C50000000000000000000000000000000000064
:103C60000000000000000000000000000000000054
:103C70000000000043000000000000000000000001
:103C80000000000000000000000000000000000034
:103C900000000000430000000000000000000000E1
:103CA0000000000000000000000000000000000014
:103CB00000000000430000000000000000000000C1
:103CC00000000000000000000000000000000000F4
:103CD00000000000430000000000000000000000A1
:103CE00000000000000000000000000000000000D4
:103CF0000000000043000000000000000000000081
:103D000000000000000000000000000000000000B3
:103D10000000000043000000000000000000000060
:103D20000000000000000000000000000000000093
:103D30000000000043000000000000000000000040
:103D40000000000000000000000000000000000073
:103D5000000000004D300008552900080000000058
:103D6000BD3A0008CC320008A8330008A833000888
:103D7000A8330008A8330008A8330008A8330008B7
:103D8000A8330008A8330008A8330008FFFFFFFF8E
:103D9000FFFFFFFFFFFFFFFFFFFF00000100415398
:103DA000434949000000000000000000000000003E
:103DB000000000000000000000000000000041536F
:103DC000434949000000000000000000000000001E
:103DD00000000000000000000000000000000000E3
:04000005080004A546
:00000001FF
